:1000000019C033C032C031C030C030C03BC02DC079
:100010002CC02BC02AC0ADC228C027C026C025C016
:1000200024C0E2C349C200C231C21FC01EC01DC0ED
:100030001CC01BC011241FBECFEFD2E0DEBFCDBF5E
:1000400011E0A0E0B1E0E2E0FBE002C005900D921B
:10005000A630B107D9F712E0A6E0B1E001C01D92C9
:10006000AB32B107E1F718D04BC5CACF1F920F9240
:100070000FB60F921124109214010F900FBE0F9023
:100080001F9018951F920F920FB60F9211240F9088
:100090000FBE0F901F901895CFEFD2E0DEBFCDBFFF
:1000A0001A9901C032C75AD06FD07BD092D388E161
:1000B0008093600087E080936000789480910001D5
:1000C000882319F010920001D0D080911401882368
:1000D00099F1F89484D342D09FD13ED1909164009D
:1000E0008FEE8093640080E480936D0084E08BBB8E
:1000F00080916800846080936800A89580EC80936C
:10010000600083B7817F846083BF83B7816083BFD2
:100110007894889583B78E7F83BFF89410926D0092
:1001200080E8809360009093640053D310923A016A
:1001300081E080930001789480913A018111B2D0DE
:100140008091D301882309F4B9CF80911901A1E0EE
:10015000B0E0082EC9D41092D301B0CF15B883E116
:1001600084B918B88FE087B91BB886EA8AB985E0E8
:100170008093C40080E48093C0001092C10010926C
:10018000C20010926F000895A0E0B0E0A5D4802DC9
:10019000992780931601883018F084E08093160127
:1001A00008959AE59093D7018091D7018093D60165
:1001B0008091D6018093D5019093DA018091DA0184
:1001C0008093D9018091D9018093D80180EF8093E9
:1001D000DC018091DC018093DB011092170181E04A
:1001E000809318011092DE019FEF90931901809186
:1001F00087018093DD019093DF01089520E009C01D
:1002000090E000000000000000009F5F9031C9F7FF
:100210002F5F2817A9F7089590E0E1EEF1E08191B2
:10022000980F82E0E932F807D1F79195909329026F
:1002300008951F93E0D05D9A80E000008F5F8F3FAC
:10024000E1F720E010E006C0822F992787709070B8
:10025000892B19F4110F489911602F5F2134A0F3F5
:10026000DBD0812F99271F91089580E090E0ADE2C7
:10027000B1E0EAE1F1E08D93119201968D309105A4
:10028000D1F7CAD0B8D059D080E48093C000109282
:10029000C1001092C20080E290E0909389008093A8
:1002A0008800089540912A0130913C0120913B0142
:1002B000EAE1F1E0ADE2B1E05CE98081853674F01D
:1002C0009C91F894935F01C099559935E8F778941B
:1002D000941710F03917A8F79C935083222389F4C0
:1002E0008C91841728F0381718F08081865F08C039
:1002F0008081181614F4815003C0882311F08F5F99
:1003000080833196119681E0E732F807B1F6222317
:1003100019F481E080933B0108958091D2019927DF
:1003200001966DE070E0B1D38093D201EDE2F1E08F
:10033000E80FF11D80819927089510928500109291
:1003400084001092800082E08093810086BB8093BD
:100350006F0010920801089510926F0082E086BB32
:1003600008951092850010928400109280001092DF
:10037000820082E086BB10926F0083E08093810050
:10038000109208010895382F299A59985C9841983D
:1003900060FF07C080911601880F8167232F255EBB
:1003A00011C020E090EA5C9897FF02C0599A01C002
:1003B00059985C9A2F5F293011F0990FF4CF232FB1
:1003C000245E84E35C989927982F88272068820F01
:1003D000911D20E05C9897FF02C0599A01C059987E
:1003E0005C9A2F5F203119F0880F991FF3CF5C982A
:1003F0005998419A0895299A5A9A419A5D9828984D
:100400005C985998549A0895299A419A5D98289829
:100410005C985998549A08955D98289829985A9804
:1004200041985C98599808951F920F920FB60F92B9
:1004300011242F938F939F93EF93FF9320912A0280
:10044000273011F429980CC0243551F480912902E9
:100450009FE089278093C60088E48093C10009C08B
:10046000E22FFF27EB52FE4F80819FE08927809388
:10047000C6002F5F20932A02FF91EF919F918F91E9
:100480002F910F900FBE0F901F9018951F920F92F3
:100490000FB60F9211248F9380E48093C0001092C6
:1004A000C1001092C20028984198299A8F910F900C
:1004B0000FBE0F901F9018951F920F920FB60F92BC
:1004C00011242F933F938F939F93EF93FF9320914A
:1004D000D1013091C6008FE038272430E9F48091B3
:1004E0000601E0910101F0910201E80FF11D308356
:1004F0008F5F809306019091D401930F9093D40164
:10050000893451F580E48093C0001092C1001092AC
:10051000C2005D982FEF20C0233031F41092060105
:100520003093070124E018C0E22FFF27E95EFE4F59
:100530008081381729F42F5F82E0809313010CC06B
:10054000223039F43F3F29F481E08093130123E006
:1005500003C01092130120E02093D101FF91EF918D
:100560009F918F913F912F910F900FBE0F901F90F1
:1005700018951F920F920FB60F9211242F933F934D
:100580004F935F936F937F938F939F93AF93BF939B
:10059000EF93FF93809108018F5F80930801815052
:1005A000823009F4BDC0833030F4882359F08130A3
:1005B00009F0F8C09AC0833009F4D3C0843009F040
:1005C000F1C0DBC080E48093C0001092C1001092A3
:1005D000C2001ADF80913B018F5F80933B019091B5
:1005E000D1019F3FB9F58091D401882399F55F9A95
:1005F00090933A0181E080932C0140910701809112
:10060000D201992701966DE070E03FD2282F332761
:10061000D901A35DBE4F8C91481751F0493540F484
:10062000F901E65EFE4F808187FD02C04C93108287
:100630002091010130910201809103019091040108
:1006400090930201809301013093040120930301F0
:10065000DCD11FC010922C0180913A018823C9F08F
:1006600080913A01815080933A0180913A01882328
:1006700041F45F9881E08093000110926F0082E066
:1006800086BBE091D201FF27E65EFE4F80818F5F3F
:1006900080838091870141DE80938701809187016B
:1006A0008093DD018091D201992701966DE070E081
:1006B000ECD1FC01E35DFE4F80818093E0018091ED
:1006C000870161E060DE80E48093C00088E0809371
:1006D000C100809188009091890084589E4F90932A
:1006E00089008093880080D15DC0809188009091BE
:1006F00089008C5B9A4F90938900809388001092B8
:100700002A0286E48093C200289A88E28093C1007E
:1007100085E58093C6008093C60078947DDD42C055
:1007200073DEA1D080918701F8DD809387018091ED
:100730008701809317011092D1011092130110923A
:10074000D4018091870160E01EDE80918800909145
:1007500089008B5D9E4F9093890080938800549808
:1007600021C08091880090918900895A9F4F909371
:100770008900809388005D9A15C01092D40180E4AE
:100780008093C00080E98093C10086E48093C2001A
:1007900080918800909189008C5B9A4F909389009A
:1007A000809388008091080165E063D190930801EF
:1007B000FF91EF91BF91AF919F918F917F916F9139
:1007C0005F914F913F912F910F900FBE0F901F900F
:1007D000189580EC8CBD5F984298409808951CBC99
:1007E0005F984298409808951F920F920FB60F920B
:1007F00011248F939F93EF93FF9380911001E82F23
:10080000FF27EF51FE4F9EB59083409A8F5F8093F4
:100810001001909111019F5F9093110191508630CA
:1008200071F48091E10180FF03C087E280931001A1
:1008300080911201882319F49E5D9093110180919B
:100840001101E0910E01F0910F01E80FF11D80817F
:100850008EBD4098FF91EF919F918F910F900FBEA9
:100860000F901F901895CF93DF9310921001109264
:100870001101A0910301B0910401B0930F01A09365
:100880000E0180913A01882379F4ED01298190913C
:10089000E2019695822F82958F70892780FF42C052
:1008A00080E1282729833EC080912C01882341F0D4
:1008B000FD018181887080930D0110920C010FC0A1
:1008C00080910C01882341F010920D01FD013196B9
:1008D000ED012981247010C081E080930C01FD019D
:1008E0003196ED019981292F247080910D01882383
:1008F00019F09460998303C080818B7F808320935B
:100900000D0180912C01882329F08C9181708093B6
:10091000120108C090E080911201882309F491E04F
:10092000909312018C918EBD429ADF91CF910895E0
:1009300080910901882329F08091E20180628093EF
:10094000E2018091E201E0910301F09104019181C3
:10095000869592959F70982790FD10C080913A01DE
:10096000882309F040C08091E301863BE1F5809146
:10097000E20192E089278093E20108958091E301EA
:10098000853B71F1863BD9F0883869F58091E501A6
:100990002091E401821738F1893518F088E58093B9
:1009A000E5013091E501832F9927821B9109853557
:1009B0009105CCF420932A0130933C010895809155
:1009C000E401809319018093DF018091E501882380
:1009D00021F081E0809309010895109209010895A2
:1009E0008FEF8093DF010895429880910B01882357
:1009F00029F08091E20188608093E2018091E20118
:100A0000847080930B0194DF0895E0910301F091CD
:100A1000040191818091E201969582958F708927DA
:100A200080FF26C09F012E5F3F4F109209018281F7
:100A3000853041F0863BE1F48381809319018093F6
:100A4000DF01089590910A01E92FFF27E051F14F4E
:100A5000D90120E084918D932F5F31962430D1F716
:100A6000892F992704966CE070E00FD080930A01DB
:100A70000895991B79E004C0991F961708F0961BFA
:100A8000881F7A95C9F78095089597FB092E072648
:100A90000AD077FD04D00CD006D000201AF470954F
:100AA00061957F4F0895F6F7909581959F4F089532
:100AB000AA1BBB1B51E107C0AA1FBB1FA617B70784
:100AC00010F0A61BB70B881F991F5A95A9F78095A0
:100AD0009095BC01CD010895F999FECFB2BDA1BD9D
:100AE000F89A119600B40895F999FECFB2BDA1BD50
:100AF00000BC11960FB6F894FA9AF99A0FBE0895B1
:020B0000FFCF25
:060B0200013D0188010025
:0C0EF000C8030900C9710904CA00000011
:00000001FF
